:030000000219FDE5
:03000B000200A848
:03002B0002015A75
:03005B000202E5B9
:030073000202D2B4
:1000800002030406080C10182030406080040608A3
:100090000C10182030406080A0C00003070F1F051F
:1000A000050D050305030302C2AFC0D0C0E0206206
:1000B00014E5256009E473E525F4F58AD262D0E001
:1000C000D0D0D2AF3285268AC262E526F4602F30C6
:1000D000682520720DD0E0D0D0D295D293D297D29D
:1000E000AF32D295D293D297206F0C206509740657
:1000F000D5E0FDE57B4290D0E0D0D0D2AF32758A1A
:1001000000C28DD26201F701B7306805206502C2D6
:100110009501B7306805206502C29701B7306805C0
:10012000206502C29301B7C29430680A2065077443
:1001300006D5E0FDC29501B7C29630680A20650772
:100140007406D5E0FDC29701B7C29230680A2065F7
:10015000077406D5E0FDC29301B7C2AFC2AD53E646
:10016000EFC0D0C0E0D2D3D2AFC2CEE52A60072024
:100170007449152A21BB7800790020742EE580305F
:100180007E01F430E50278FF53DACF207E0343DAB4
:1001900020307E0343DA10C2D8C271E580307E0180
:1001A000F430E50279FFC3E89970CB306103752A1A
:1001B00018207403752A18885CD27020740DE52B02
:1001C0006004152B21CB43DA01C2D8207002413ED6
:1001D000A85C206102C270207431C3E894F040032F
:1001E00074F0F8E8C4540F28F87984B70302410B7F
:1001F000C313C3138721200802C313200A06C3C8F0
:1002000098F8410B28F8500374FFF8C3E89565503F
:1002100003E565F88822E52D54066022206B1FE572
:1002200036C333C333F8E564C313C313F9C395224C
:1002300040028922E82522F52250037522FF8522FB
:1002400024A824C3E52495614002A8618825E566B9
:1002500070024182C3E8AA669A5003E8FAE4F9EA18
:10026000C333FBE568F45B29400D2567F8E567605B
:10027000021567400B41820AC3E5679A5002056781
:1002800078FF8826C26FC3E52694F84002D26F201B
:10029000CF0AD0E0D0D043E610D2AD32C2CF053A7B
:1002A0007801E52A6005307402152AC3E55C9401E3
:1002B0004005755F0041C8756000756900E55F2401
:1002C00001F55F5003755FFFD0E0D0D043E610D258
:1002D000AD32C2AF53E67F7592FA7593FFC2607577
:1002E0009104D2AF32C2AF53E6EFC2ADC0D0C0E08E
:1002F000C0F0D2D3D2AFA8FBA9FCC2D83071026142
:100300004C53DACF207E0343DA10307E0343DA20E9
:10031000D271E580307E01F420E5026123882789CF
:1003200028A17953DACF207E0343DA20307E0343BD
:10033000DA10C2D8C271307402A1657800E580304D
:100340007E01F430E502A165885CA14D53DACF202F
:100350007E0343DA20307E0343DA10C2712061024B
:10036000812553DACF207E0343DA10307E0343DA4F
:1003700020C2D8D27188578958C3E89555F8E995B5
:1003800056F97B007E087A00C3E8948CE99400500B
:1003900005755B008117882178A2E6A8216055C306
:1003A000E894C8E994005008E4D2E4FB7A0A61F2C8
:1003B000C3E89468E994015008E4D2E3FB7A0F6142
:1003C000F2C3E894D0E994025008E4D2E2FB7A1E2A
:1003D00061F2C3E894A0E994055008E4D2E1FB7A05
:1003E0003C61F2C3E89498E994085008E4D2E0FB39
:1003F0007A787E00C3E89559FCE9955AFD30E70A02
:10040000ECF42401FCEDF43400FD755B00C3EC9AC0
:10041000ED9E5003755B018859895A85575585585B
:10042000567802A14DC3E89527F8E99528F9307C64
:1004300002A131307B02A131307A02A12A2075025B
:100440008148E9FDE8FC8167E9C313F9E813F83056
:100450007902A12AE9C313F9E813F8307802A12A36
:10046000E9C313FDE813FC20612CC3EC941CED944C
:0E047000024002817EED701EC3EC94C850184D
:10047E000529E52970021529C3E529940A5002A120
:10048E0065755C00D270A165E52960021529788832
:10049E00E6F97400207F087896B90302789EE62468
:1004AE00FAFEE43400FFC3EC9EFCED9FFD9208B90A
:1004BE000310A2085007207609D27681D03076023A
:1004CE00C276A2085016B9030DECF42401FCEDF42B
:1004DE003400FD0204EA78007900A131B90315EC6D
:1004EE0033FCED33FDC3EC940AFCED9400FD500497
:1004FE007C007D00C3EC94FFED9400400678FF79FC
:10050E0000A131EC8572F0A4C5F0A2F733F87900A2
:10051E00400302054D78FF790002054DE9C313F93A
:10052E00E813F8307C0EE9600278FFC3E81338F860
:10053E00E43400F9C3E894FFE99400400278FF88A0
:10054E005CD270206102A165741FF4552F4BF52FFC
:10055E00C274EB7002D274752A18307403752A0AAD
:10056E00306102A17920740353DAFE207403752BD7
:10057E0006D0F0D0E0D0D0D2AD43E61032790102F1
:10058E0005A979030205A9790A0205A9791E0205B2
:10059E00A979640205A979C80205A97817E4D5E0FE
:1005AE00FDD8FAD9F6227A147B780205D07A107B20
:1005BE008C0205D07A0D7BB40205D07A0B7BC80273
:1005CE0005D0E573D5E001227902E4C296D5E0FDAF
:1005DE00C297D5E0FDD297D5E0FDD296D5E0FDE9E4
:1005EE0020E002C29530E002C293E573D5E0FDE94A
:1005FE0020E002D29530E002D2937496D5E0FDD978
:10060E00C9EAF8D5E0FDD8FBDBB8C29622C37C0060
:10061E007D0075F00005F0EA33FAEB33FB50F6EB94
:10062E0013FBEA13FAC3E9FFE8FEE89AF8E99BF92F
:10063E005004EFF9EEF8B3EC33FCED33FDD5F0DFFB
:10064E00EDF9ECF822E889F08A20D2D4F8A9F07BF3
:10065E000030F70B7BFFF42401F8E9F43400F9E8DD
:10066E008520F0A4ADF0F8E98520F0A4AFF0FEED02
:10067E002EF974003FFA7C04C3EA13FAE913F9E881
:10068E0013F8DCF48BF030F70AE8F42401F8E9F4FF
:10069E003400F9E889F0C2D4F8A9F02222C3E5416A
:1006AE0013F9E54013F8C3E54498F8E54599F95078
:1006BE000CC3E89480E994FF40160206E2C3E89466
:1006CE007FE9940050030206E2787F79000206E289
:1006DE00788079FF8849894A22E5492546F8E54A16
:1006EE003547F9854A20E4300701F43548FA30E7FA
:1006FE0009C3EA94F04015020720C3EA940F500391
:10070E0002072078FF79FF7A0F0207207800790020
:10071E007AF0C3E5249561500AC374019524500BF9
:10072E0002073EE54A20E70E02073EE54A30E7069D
:10073E00884689478A482278A5E6FAC3E54933F800
:10074E00E54A33F9D153E930E70BC3E89480E994D5
:10075E00FF4013E178C3E8947FE994005002E178FA
:10076E00787F7900E178788079FFE820E715C3E596
:10077E002398F84009C3E89401400302079F7801CB
:10078E0002079FE8F424012523F8400302079F780F
:10079E00FF884B2278A6E6FAA847A948D153E9303C
:1007AE00E70CC3E89401E994FF40160207D3C3E8AF
:1007BE0094FFE9940050030207D378FF79000207F3
:1007CE00D3780179FFE920E715C3E54B98F8400986
:1007DE00C3E8940140030207FA78010207FAE8F42D
:1007EE002401254BF840030207FA78FF882422786B
:1007FE00FF20692879A1E76023E541601F74FF851A
:10080E0041F0848539F0306A0375F005A4F8C5F01F
:10081E00600278FFC3E895645002A864886322C31F
:10082E00E5409440E5419401E563500314013E0414
:10083E006002F563220208462275E890227883E66C
:10084E00FF30EDF9A8BDA9BE0570C3E57094084050
:10085E0052757000E9FA79A0E76044EA7007E57115
:0F086E00601B02087FC3E895716010E5715006AA
:10087D00600C1402088B0460F902088BE571F571A8
:10088D00C3946D401B7561C0C394044013756180A2
:10089D00C39404400B756140C3940440037561001B
:1008AD0075BB0822E561F460020561E570B40703CC
:1008BD0075BB1022743279A787F0A4C5F0A2F73367
:1008CD00F8C3E895614002A86188228824882588AC
:1008DD00268864227540007541F022C2AF75C8208C
:1008ED00A8CCA9CDAA3A30CF010A75C824D2AFAB96
:1008FD003BAC3C883B893CC3E89BF8E99C206908EC
:10090D00F930660221F72151AD3D8A3DF9EA9DFA94
:10091D00600478FF79FFAE3EAF3F8B3E8C3FA83B26
:10092D00A93CC3E89EF8E99FF9C3E54113FBE540F7
:10093D0013FAE82AF540E93BF54150067540FF757D
:10094D0041FF219EAA40AB41AC40AD417E047F02E8
:10095D00C3EB9404400D1E1FC3EB94084005206AA1
:10096D00021E1FC3ED13FDEC13FCDEF7C3EA9CFA68
:10097D00EB9DFBEF6009C3E913F9E813F8DFF7EA24
:10098D0028FAEB39FB8A408B4150067BFF8B408B5D
:10099D0041C3EB94025002D2663069047F0321C932
:1009AD007892E6FFC3E537948240110FC3E5379483
:1009BD00A040010FC3EF940640027F057E02E54182
:1009CD00C4540FF9E541C454F0F8E540C4540F2860
:1009DD00F8C3E89EFAE99400FB4009C3EA9402EBE0
:1009ED00940050047A02E4FB4143AA40AB41EBC4AE
:1009FD00FEEAC4540F4EFCC3EA9CFAEB9400FBC311
:100A0D00E813C313F8EA28FAEB3400FB8A408B4154
:100A1D00C3EB94024002C2667802EBC4FE7B00EA8F
:100A2D00C4540F4EFAC3EA98FA4005C3940250021B
:100A3D007A027892E6FF30600241438551928552E9
:100A4D0093D26043E680C3E49AF8E49BF9306602E2
:100A5D0041CFE8FAE9FBD3E913FDE813FC8851898E
:100A6D0052C3EF94036038EF20E00DE82CF8E93D18
:100A7D00F9ECFAEDFB020A98E828F8E939F9C3E830
:100A8D002402F8E93400F97AFE7BFFC3EF940340AA
:100A9D000E8A538B54884D894E8C4F8D506103882F
:100AAD005389548A4D8B4E8C4F8D5030691275532E
:100ABD00F07554FF754FF07550FF7551F07552FF7D
:100ACD006103E8FAD3E813FC8851C3EF9403602067
:100ADD00EF20E007E82CF8ECFA41EFE8282402F8C3
:100AED007AFEC3EF940340088A53884D8C4F6103FF
:100AFD0088538A4D8C4FE568C3335002646BF5689B
:100B0D00306002610D753402D26043E680E52D54EC
:100B1D00066034A840A941C3E913F9E813F8C3E905
:100B2D0013F9E813F8306904E92440F9C2AF53E62C
:100B3D007F759100C3E498F594E499F5957591044A
:100B4D00D26043E680D2AF22D26475430075200097
:100B5D00306C03752040020B74D264754300752010
:100B6D0040306C0375200078017901206620E52D59
:100B7D0054066002C2647914E541C313700104F890
:100B8D00C3941440027814306904781B791B2060DB
:100B9D0010E543600C306903D53404D26D811E71AC
:100BAD00150543E59B5440B52002810830690908BD
:100BBD00C3E899400118619B20640A08C3E8994075
:100BCD00026174619BC264C2AF53E67F75910030C0
:100BDD0066127594007595F8759104D26043E680A0
:100BED00D2AF6174E5417EFFC3334005C33340018D
:100BFD00FEC3E49E759400F59561E5C3E53394015C
:100C0D00500261743064026174D802811C619BC210
:100C1D006DC2AF53E67F75910085539485549575DC
:100C2D009104854D92854E93D26043E680D2AFE517
:100C3D002D54066008206A020533020C5A306D0DE2
:100C4D00206C0A2064071581158102151D2278007C
:100C5D003064027801E53775F007A4F9E5F028F561
:0E0C6D00F0E9A2F013A2F113A2F213F537C3BF
:100C7B0094785003753778C3E53795384008D265BB
:100C8B00D295D293D2973060028191854F92855045
:100C9B0093D26043E68022207D16C2AF754202C21A
:100CAB0096D294306202C293D2AF759F11020E910D
:100CBB00C2AF754202C296D292306202C295D2AFD7
:100CCB00759F11020E91307243207D20C2AF754289
:100CDB0003900138757B40D293C292306204C29765
:100CEB0081EFD296D2AF759F13020E91C2AF7542B0
:100CFB0003900138757B40D295C294306204C29741
:100D0B00A10FD296D2AF759F10020E91207D17C204
:100D1B00AF754203900113D293306202C297D2AFE8
:100D2B00759F13020E91C2AF754203900113D295BA
:100D3B00306202C297D2AF759F10020E91207D16C2
:100D4B00C2AF754204C294D292306202C297D2AF44
:100D5B00759F10020E91C2AF754204C292D29430AD
:100D6B006202C297D2AF759F13020E91307243206D
:100D7B007D20C2AF754205900127757B10D297C2BB
:100D8B0096306204C295A195D294D2AF759F110291
:100D9B000E91C2AF754205900149757B04D297C283
:100DAB0096306204C293A1B5D292D2AF759F110255
:100DBB000E91207D17C2AF754205900109D2973075
:100DCB006202C295D2AF759F11020E91C2AF7542EE
:100DDB000590011DD2973062EBC293D2AF759F1174
:100DEB00020E91207D16C2AF754206C292D296308A
:100DFB006202C295D2AF759F13020E91C2AF7542BC
:100E0B0006C294D296306202C293D2AF759F100283
:100E1B000E91307243207D20C2AF75420190014983
:100E2B00757B04D295C294306204C293C13BD292BB
:100E3B00D2AF759F10020E91C2AF75420190012780
:100E4B00757B10D293C292306204C295C15BD2946F
:100E5B00D2AF759F13020E91207D17C2AF75420161
:100E6B0090011DD295306202C293D2AF759F1002D2
:100E7B000E91C2AF754201900109D293306202C24A
:100E8B0095D2AF759F13C26522900107757B00D277
:100E9B0095D293D297C294C292C296C262227880A4
:100EAB0076FF0876FF0876FF0876FF08760308764C
:100EBB000408760A087603087601087601788C76A2
:100ECB00010876FF0876FF0876FF0876FF0876FFA5
:100EDB000876030876FF0876FF0876FF0876250864
:100EEB0076D00876FA0876FA0876040876FF087644
:100EFB000108760008767A0876FF087601087601F5
:100F0B00087600087603087600227887E6FFC2721F
:100F1B00BF0302D2727888E6C394036008C27DE6F1
:100F2B0030E102D27DC27E7889E630E102D27EC307
:100F3B00EF94026008758E01D273020F4D758E000F
:100F4B00C273227880E6149000809378A5F678819E
:100F5B00E6149000809378A6F67886E61490008DC0
:100F6B009378A7F67886E6F539C394025003753962
:100F7B0002789CE67538FFB402037538A0B40303FE
:100F8B0075388278A3E61490009A93F566D1942273
:100F9B00227896E6FA7897E6FB7888E6B40305C3E1
:100FAB00EB940EFB307F047A007BFFC3EB9AFCC300
:100FBB00948250027C827572000572EC8572F0A4EB
:100FCB00C3E5F0947D40F222D27FF19C12059A1278
:100FDB00059A7A007B007C10120590E55C2AFA7466
:100FEB00003BFBDCF37C04C3EB13FBEA13FADCF7EB
:100FFB00FEC27F120F9C22757C00757D00E5EF20F1
:10100B00E6037520000520903FFFE5201460069055
:10101B001DFF1460009304600375EF1653D9BF7561
:10102B0081C043FF8012058B75EF0643B203E5B316
:10103B00240220E70DF521E5E320E0068521B343EB
:10104B00E301120E947580FF75A40075F1B275D48F
:10105B00DF7590A975A5FC75F2FE75D50175A60116
:0E106B0075E241120E94E4F8F6D8FD756801A6
:10107900120EA912156E78988673753001C2AF12D7
:1010890005A41205B412059A1205BB12059A120598
:10109900C212059A12168B1205A41205A412059FF5
:1010A900C2AF757C00757D0078FA79FA308507D969
:1010B900FBD8F7021C00120F15120F4E120F9B12CC
:1010C9000F9C78988673120E94758810758902752D
:1010D900C82475910475D84075A82275B80275E6BB
:1010E90090759B80759D0075D10E75BC5875BB08B0
:1010F90075BA1175E88012058BD2AF12084375369F
:101109000053DACF207E0343DA20307E0343DA101E
:1011190043DA01C2D8C2711205A4D2617B037A0CE9
:10112900E55B70077A0CDB030210A912059A20709F
:10113900030210A9C270E55CC3940240E1E52F5493
:101149001F855E5DF55EB55DD5DAD5C26153DACF2F
:10115900207E0343DA20307E0343DA10C2D8C271FD
:1011690078A2E67008D274E52F54E0F52FC27575A0
:10117900290012059F307409C3E529940A4002D257
:101189007512059078023074027800C3E55C9840C6
:10119900F0C2AF1205B41205B41205B4D2AF1205EC
:1011A900A4754C007888E6B4030241A91205907829
:1011B9008CE6C3940150030212A9E530C39401508F
:1011C900030212A9757CA5757DF1207435C3E55C10
:1011D90094FF50030212A9C2AF1205C9D2AF12057A
:1011E9009FC3E55C940150EFC2AF1205B412059597
:1011F9001205B4D2AF12059FC3E55C94FF40E90222
:1012090017107F05D27F120F9C12059FC2AFC27FB4
:10121900120F9CAE5CC3E55C947FD2AF500241B91A
:1012290012058BC2AF1205C9D2AFDFD8120FD3C3D3
:10123900EE94057897F61205A41216937F0AD27FC9
:10124900120F9C12059FC2AFC27F120F9CAE5CC3E6
:10125900E55C947FD2AF50E412058BC2AF1205B49E
:101269001205951205B4D2AFDFD4120FD3EE2403C1
:101279007896F6F87997E7C394824003985006E880
:1012890024827897F61205A41215B01216C2120517
:101299009F120F9CC3E55C94FF500221CD021710E9
:1012A900757C00757D00C3E55C954C4003855C4CFD
:1012B90012059F78017988E7B403027805C3E55CD4
:1012C90098400221ADC2AF1205C91205C91205C95C
:1012D900D2AF1205A4753000E4F531F5320531E5D8
:1012E90031F4703F0532789AE67819146012783231
:1012F90014600D787D14600878FA14600375320063
:10130900C3E53298401D120E9412058B15327531C2
:101319000078998673C2AF1205C9D2AF78988673DF
:1013290012059F120595E52A700530740201A97806
:10133900012074027806C3E55C9840A17888E6C369
:101349009403600312059FE52A70030210A9C2AF36
:10135900120E94E4F522F523F524F525F526F56713
:10136900D2AF7885E6C333F565E4F544F545F5462E
:10137900F547F548F570F52CF52DF53775700875B5
:10138900BB1012058B12084730EDFDA8BDA9BEE9B7
:101399007001F8887112084B75700875BB10120F2F
:1013A90015C2AF7561FF1208C18522618522628568
:1013B9002263D2AF752201752401752501752601B5
:1013C900856069756A017888E6B40307C27D30765D
:1013D90002D27DD268D269753300120DEE120E1D4C
:1013E9001208E11208E81208E11208E81208E112ED
:1013F9000B661206AA120C5B120CA21208E8120B59
:1014090055306E031206AB2066031207FD306603E2
:1014190012082D120C5B120CD11208E8120B66305F
:101429006E031206E7120C5B120D481208E8120B44
:1014390055306E03120745120C5B120D771208E83E
:10144900120B66306E031207A2120C5B120DEE121C
:1014590008E8120847120B55120C5B120E1D1208F0
:0D1469004B1208E830692F856461856462CC
:10147600856069756A0179187A0CC3E53399400C61
:10148600C269D26A8A357561FF02149FC3E55C940E
:101496000140030213F8021525306A1D206C1AE577
:1014A60035147006C26AD26B61F8F535C3E55C94F3
:1014B6000140030213F8021525753600788279A4D7
:1014C600E760027803C3E55F985054307404E52A58
:1014D600604D7888E6B40317207D0520760781F5F0
:1014E60030760281F5206C07D26C8564618137788D
:1014F600F0306C058564617820C3E541985002613F
:10150600F8306C1BC26CC27D307602D27DD26A7511
:10151600351285646161F80536E55C6002A12875BF
:101526003600C2AF120E947887E6FE7602120F15C9
:101536007887EEF6E4F522F523F524F525F526F56C
:1015460065752C00752D00D2AF12059F120E94788A
:10155600A4E66006C295C297C293307409C3E53605
:101566009404400201A941E1901A0D78201215F267
:10157600E520B45A0CA31215F2E520B4A503021512
:1015860090120EA91215B00215AF901A0378807B3F
:101596000A1215F2A308DBF9901A0F788C7B191240
:1015A60015F2A308DBF9901A2822C2AF12163512DB
:1015B6001612901A00740E1215F7A374071215F777
:1015C600A374151215F7901A0378807B0A1215F684
:1015D600A308DBF9901A0F788C7B191215F6A3086D
:1015E600DBF9121648121626901A2822E493F622E0
:1015F600E6438F01538FFDFFC3E583941C40012210
:10160600EF857CB7857DB7F0538FFE22438F02436B
:101616008F01857CB7857DB7901A0DF0538FFC221C
:10162600901A0D745AB1F7901A0E74A5B1F7227A72
:101636003079D07820901A40B1F2E520F709A3DA84
:10164600F7227A3079D0901A40E7B1F709A3DAF990
:1016560022AB74A875BB01027984BB02027985BBF3
:1016660003027986BB04027992BB05027987BB0621
:101676000279A3BB0702799CBB08027988BB0902E1
:101686007989E8F7227C051205A4DCFB22C2AF1299
:1016960005B41205BB1205C21205C912059512053D
:1016A600B41205BB1205C21205C91205951205B47E
:1016B6001205BB1205C21205C9D2AF22C2AF12056E
:1016C600C91205C21205BB1205B41205951205C949
:1016D6001205C21205BB1205B41205951205C912F0
:1016E60005C21205BB1205B4D2AF22AE74AF75C2E5
:1016F600AF1205B41205B41205B4120595DEF21246
:1017060005C9120595DFF8D2AF22D193D18BD18BC3
:10171600757401757501757600D1F17C05AD5C12A5
:1017260005A4C3ED955C70F5C3E55C9401400AC35E
:10173600E55C94FF403202174CD157B1B0D193C249
:10174600AF75EF16D18BDCD50576C3E576940350DD
:101756000280C6D18B0575E5741490009F93F80836
:10176600C3E57598500280AED18BD18B0574C3E565
:1017760074940A5002809C120EA9B1B0C2AF75EFE4
:0317860016D18BEE
:0319FD00021002D3
:101A00000E0715FFFFFFFF03040A0301015AA5019A
:101A1000FFFFFFFFFF03FFFFFF25D0FAFA04FF01DE
:091A2000007AFF0101000300FF40
:101A4000235475726E6967794E6665743235412329
:101A500023424C48454C4923463333302320202031
:101A60002020202020202020202020202020202076
:101C0000C2AFC2D353D9BF7581C043B20343FF8073
:101C1000752438752503B1DC7529A5752AF175E29F
:101C20004043F12053A4DF75D4FFD2857DFA7803B9
:101C300079E67C10752200752300901DE97B0675FE
:101C400024987525013085028145208508D8FBD967
:101C5000F9DCF781B7308508D8FBD9F9DCF781B713
:101C6000B19CE493A3C39A6004DDC381B7DBDBB10D
:101C70008E6002812E7B08E493FAA3B16FDBF87AC1
:101C800030B16F752200752300B18EEAFCEBFDC305
:101C9000ED94FE400EB18E8A278B28ED30E0048A49
:101CA000828B83B18E7AC270D8C3ED94FE601950D6
:101CB000CEBD002BEC600F7520007521FF7529004B
:101CC000752A000200008100A827A9280809D80465
:101CD000D90281DCB192EA89AAF281CE0D81A3C337
:101CE000ED94035053EDA2E092007AC5C3E58294CF
:101CF00000E583941C508A200010438F02438F011B
:101D00008529B7852AB7F0300029A827A92808090E
:101D1000438F01538FFDD804D902A133C3E58394C7
:101D20001C4003A3A11689AAE28529B7852AB7F02A
:101D3000A3A116538FFC817F7AC1BD030CE493A34A
:101D4000FAB153DCF8B14B817F8181AA22AB23B178
:101D50006FEBFAEA6222752608C3E52313F523E543
:101D60002213F52250066323A0632201D526EAB18F
:101D7000DCB1DC75260AEAF4200102D285300102CA
:101D8000C285B1DCC3134002C201D526EB22B19259
:101D9000EAFB208502A192308502A197752608AE44
:101DA00024AF25C3EF13FFEE13FEB1E0B1DCC3EAAD
:101DB000133085024480FA30E703632201C3E52330
:101DC00013F523E52213F52250066323A0632201B5
:101DD000D526D9E52265236523F52222AE24AF2539
:101DE0000E0FDEFEDFFCD20122424C48656C6934E6
:071DF000373163F3300601F7
:00000001FF
